:10000000D33084000730FE001330FF001120800041
:10001000840A0408D73A03191528FF0A0319FE0AAF
:1000200006287E088A007F088200683084007030CD
:100030000A128A1132200A128A11D7308400F03055
:100040000A128A1132200A128A1183177130840031
:100050007E300A128A1132200A128A1183010A1292
:100060008A113A2864008001840A040603190034C6
:100070000406332883160313FF3085000310831210
:1000800003130030031801308500031000300318FB
:1000900001309F000630831603139F0003100030C9
:1000A0000318013086000310831203130030031875
:1000B00001308600031000300318013087008130C2
:1000C00083160313870083120313101690169010E3
:1000D00064300A168A152C250A128A110A168A110A
:1000E00002220A128A1164300A168A152C250A1275
:1000F0008A110A168A155E240A128A1164300A16B9
:100100008A152C250A128A1180300A168A15522463
:100110000A128A1164300A168A152C250A128A11CD
:100120008E3083120313AB000630AC000A128A1122
:100130003F220A128A11C0300A168A1552240A1266
:100140008A11AF3083120313AB000630AC000A12E1
:100150008A113F220A128A11FA300A168A152C25B2
:100160000A128A110A168A155E240A128A1164304C
:100170000A168A152C250A128A1180300A168A1549
:1001800052240A128A11FF3083120313AB00063087
:10019000AC000A128A113F220A128A11043083121B
:1001A0000313A0002008A5000030A4000030A30025
:1001B0002530A2008030A10004300A128A150020E8
:1001C0000A128A11633083120313A2000630A300BF
:1001D0000A168A15CF250A128A1100300A168A15C6
:1001E000AB250A128A1183120313A0002008FC0019
:1001F00001300A168A15AB250A128A1183120313DD
:10020000A0002008FD000A168A159C240A128A11F3
:10021000831203132908FA01FA072A08FB01FB07D6
:100220000C307A067B04031D1629172956290A1655
:100230008A155E240A128A1180300A168A15522401
:100240000A128A11FF3083120313AB000630AC0090
:100250000A128A113F220A128A110A128A113B23BA
:100260000A128A11831203132108EA01EA072208FD
:10027000EB01EB070A168A11B2230A128A11C03069
:100280000A168A1552240A128A1128300A168A156B
:100290002C250A128A119F3083120313AB000630FB
:1002A000AC000A128A113F220A128A11033083120B
:1002B00003137A067B04031D5E295F29CB290716E9
:1002C000FF300A168A152C250A128A11FF300A16E9
:1002D0008A152C250A128A11831203138712FF3004
:1002E0000A168A152C250A128A11FF300A168A1559
:1002F0002C250A128A1183120313871500300A165F
:100300008A15B0240A128A11831203138711FF3051
:100310000A168A152C250A128A11831203138715CF
:100320008716FF300A168A152C250A128A118312A5
:1003300003138711FF300A168A152C250A128A1119
:10034000FF300A168A152C250A128A11831203130C
:1003500087150712FF300A168A152C250A128A11F2
:10036000FF300A168A152C250A128A1183120313EC
:100370008711871501300A168A15B0240A128A11CE
:10038000FF300A168A152C250A128A1183120313CC
:100390008711071687160E307A067B04031DD129B4
:1003A000D229F8290A300A168A152C250A128A1130
:1003B000EF290030A1000030A2000A168A15DC24C3
:1003C0000A128A110A168A159C240A128A118312AB
:1003D00003132908FA01FA072A08FB01FB070E306C
:1003E000831203137A067B040319F729F829D92904
:1003F0000F307A067B04031DFE29FF29252A0A30C7
:100400000A168A152C250A128A111C2A0130A1000D
:100410000030A2000A168A15DC240A128A110A1674
:100420008A159C240A128A11831203132908FA01DF
:10043000FA072A08FB01FB070F30831203137A0621
:100440007B040319242A252A062A0718282A292A80
:10045000382A87150A128A159D260A128A11FA303F
:100460000A168A152C250A128A1183120313871182
:0804700003290A128A11002879
:10047E008616572A2B0884002C080A128A11002689
:10048E000A128A110A168A1588250A128A11013053
:10049E0083120313AB070318AC0AAD00AD1BAC03FC
:1004AE002B0884002C080A128A1100260A128A11BF
:1004BE000038031D632A642A412A08000030CE004A
:1004CE000030CF000030D0003C08CB003D08CC00FF
:1004DE003E08CD000A168A15B6270A128A1103188D
:1004EE00792A7A2A872A213083120313E8000030F2
:1004FE00E9000030BC000030BD000030BE003A2BD9
:10050E008312031300303E06031D932A00303D066E
:10051E00031D932A00303C06031D962A972AA22A11
:10052E002230E8000030E9000030BC000030BD0091
:10053E000030BE003A2B3F30C1004108CE003C08CF
:10054E00CB003D08CC003E08CD000A168A110720CC
:10055E000A128A11831203134B08D2004C08D300DF
:10056E004D08D4000030D5000030D6004030D70002
:10057E000A128A155F200A128A1183120313520877
:10058E00D2005308D3005408D4000030D500803078
:10059E00D600BF30D7000A128A1530240A128A11EB
:1005AE00831203135208BC005308BD005408BE004A
:1005BE00FF30BF070318C00AFF30C0070830C7005E
:1005CE000030C8002A30C5000630C6003C08C20004
:1005DE003D08C3003E08C4000A168A1162270A129B
:1005EE008A11831203134208BC004308BD0044085D
:1005FE00BE003F08C201C2074008C301C3070A1666
:10060E008A1157200A128A11831203134208D2004C
:10061E004308D3004408D4007230D5003130D600E0
:10062E003F30D7000A128A155F200A128A118312F0
:10063E0003135208D2005308D3005408D4003C08C8
:10064E00D5003D08D6003E08D7000A128A15302480
:10065E000A128A11831203135208BC005308BD00FC
:10066E005408BE003A2B0800023083120313A70071
:10067E000030A8000030A3000030A4000030A50018
:10068E000030A600F42D871514300A168A152C2575
:10069E000A128A110A168A159C240A128A118312CA
:1006AE0003132908A301A3072A08A401A4071430E1
:1006BE000A168A152C250A128A1183120313871122
:1006CE00CE2D87152708AB01AB072808AC01AC0768
:1006DE000A30A9000030AA000A168A1524270A1229
:1006EE008A11831203132908A5070318A60A2A08DC
:1006FE00A6072508A901A9072608AA01AA070A160E
:10070E008A151E260A128A1183120313FF30A707B9
:10071E000318A80AFF30A80714300A168A152C25CC
:10072E000A128A11831203138711F42D87152708D5
:10073E00AB01AB072808AC01AC070A30A9000030AA
:10074E00AA000A168A1524270A128A11013084007B
:10075E00031083120313A90DAA0D840BAF2B2908C6
:10076E00A5070318A60A2A08A6072508A901A9079E
:10077E002608AA01AA070A168A151E260A128A1127
:10078E0083120313FF30A7070318A80AFF30A80728
:10079E0014300A168A152C250A128A118312031395
:1007AE008711F42D87152708AB01AB072808AC017C
:1007BE00AC070A30A9000030AA000A168A152427B1
:1007CE000A128A11831203132908D201D2072A08AA
:1007DE00D301D3070330D4000030D5000A168A1592
:1007EE00F4250A128A11831203135208A50703185F
:1007FE00A60A5308A6072508A901A9072608AA01D3
:10080E00AA070A168A151E260A128A1183120313C4
:10081E00FF30A7070318A80AFF30A80714300A16DE
:10082E008A152C250A128A11831203138711F42DAF
:10083E0087152708AB01AB072808AC01AC070A30B7
:10084E00A9000030AA000A168A1524270A128A1156
:10085E0002308400031083120313A90DAA0D840B1A
:10086E00312C2908A5070318A60A2A08A607250869
:10087E00A901A9072608AA01AA070A168A151E2683
:10088E000A128A1183120313FF30A7070318A80A4E
:10089E00FF30A80714300A168A152C250A128A1161
:1008AE00831203138711F42D87152708AB01AB07AD
:1008BE002808AC01AC070A30A9000030AA000A16BD
:1008CE008A1524270A128A11831203132908D201CA
:1008DE00D2072A08D301D3070530D4000030D50043
:1008EE000A168A15F4250A128A1183120313520866
:1008FE00A5070318A60A5308A6072508A901A907E4
:10090E002608AA01AA070A168A151E260A128A1195
:10091E0083120313FF30A7070318A80AFF30A80796
:10092E0014300A168A152C250A128A118312031303
:10093E008711F42D87152708AB01AB072808AC01EA
:10094E00AC070A30A9000030AA000A168A1524271F
:10095E000A128A11831203132908D201D2072A0818
:10096E00D301D3070630D4000030D5000A168A15FD
:10097E00F4250A128A11831203135208A5070318CD
:10098E00A60A5308A6072508A901A9072608AA0141
:10099E00AA070A168A151E260A128A118312031333
:1009AE00FF30A7070318A80AFF30A80714300A164D
:1009BE008A152C250A128A11831203138711F42D1E
:1009CE0087152708AB01AB072808AC01AC070A3026
:1009DE00A9000030AA000A168A1524270A128A11C5
:1009EE00831203132908D201D2072A08D301D30791
:1009FE000730D4000030D5000A168A15F4250A12E5
:100A0E008A11831203135208A5070318A60A530866
:100A1E00A6072508A901A9072608AA01AA070A16EA
:100A2E008A151E260A128A1183120313FF30A70796
:100A3E000318A80AFF30A80714300A168A152C25A9
:100A4E000A128A11831203138711F42D87152708B2
:100A5E00AB01AB072808AC01AC070A30A900003087
:100A6E00AA000A168A1524270A128A110330840056
:100A7E00031083120313A90DAA0D840B3F2D290811
:100A8E00A5070318A60A2A08A6072508A901A9077B
:100A9E002608AA01AA070A168A151E260A128A1104
:100AAE0083120313FF30A7070318A80AFF30A80705
:100ABE0014300A168A152C250A128A118312031372
:100ACE008711F42D87152708AB01AB072808AC0159
:100ADE00AC070A30A9000030AA000A168A1524278E
:100AEE000A128A11831203132908D201D2072A0887
:100AFE00D301D3070930D4000030D5000A168A1569
:100B0E00F4250A128A11831203135208A50703183B
:100B1E00A60A5308A6072508A901A9072608AA01AF
:100B2E00AA070A168A151E260A128A1183120313A1
:100B3E00FF30A7070318A80AFF30A80714300A16BB
:100B4E008A152C250A128A11831203138711F42D8C
:100B5E0087152508A901A9072608AA01AA070A16BA
:100B6E008A151E260A128A1183120313FF30A70755
:100B7E000318A80AFF30A80714300A168A152C2568
:100B8E000A128A11831203138711F42DF42DEF2DFF
:100B9E002308003A0319682B013A03199D2B033AD7
:100BAE000319D92B063A03191F2C013A03195B2C92
:100BBE00033A0319A12C0E3A0319E72C013A031933
:100BCE002D2D033A0319692D073A0319AF2DCD2D9B
:100BDE002408003A0319CF2DCD2DA81FF72DF82D7F
:100BEE004A2B2508A101A1072608A201A207FF2D65
:100BFE000800FE00FE1F082E83137E1883170008C0
:100C0E0008008A00040882000034003480343F3427
:100C1E00723431343F34FE3475343E3458346334D8
:100C2E003D3495341D343C34C534AE343A347934C5
:100C3E00213439349434803437349334A7343534F2
:100C4E0056341534343400340034003400348034D7
:100C5E003F34F034FF34BE34E234A9343E348334AE
:100C6E007634BE34AE342B343E343C34C334BD34CF
:100C7E00D23413343D347834D334BB34003400349E
:100C8E004034FF3445347834693474346534643414
:100C9E002C34203470346C346534613473346534E0
:100CAE0020347234653462346F346F3474342034CB
:100CBE0070346934633400342D342D345334653438
:100CCE007234693461346C34203469346E3469346E
:100CDE007434203463346F346D3470346C34653452
:100CEE00743465342D342D340034613464346D34F1
:100CFE0069346E344034733474347234613466340F
:100D0E0061346E347434653424343E3400345234D9
:100D1E0048344D342D343134203466346F347234CB
:100D2E00203443342E3441342E344D342E3400349A
:100D3E00203445344E3454344534523420345434F3
:100D4E004F342034533454344134523454340034F8
:100D5E002034203442347934203444342E34443414
:100D6E0061346C34203446347234613420340034AF
:100D7E00613464346A342034763461346C347534BE
:100D8E0065343A345B340034683466347434203459
:100D9E00763461346C34753465343A345B340034F3
:100DAE00773472346934743465342034683466347C
:100DBE0074342034003477347234693474346534C6
:100DCE002034613464346A3420340034723465342F
:100DDE0061346434203468346634743400347234CC
:100DEE006534613464342034613464346A340034DC
:100DFE0043346F347234733461343A3420340034F3
:100E0E006534783469347434003420346D346D3480
:100E1E00003420345D3400340D340A3430347534EB
:100E2E00AC00AB08031D1C2F1F2F1030AF00212F5D
:100E3E004030AF000030B3000030B2000030B100DF
:100E4E000230B0000030CF000F30CE004230CD0067
:100E5E004030CC002C08C400C501C601C7014708AC
:100E6E00CB004608CA004508C9004408C8000A1647
:100E7E008A15E0260A128A11831203134B08BB004F
:100E8E004A08BA004908B9004808B8002A08CF0035
:100E9E002908CE002808CD002708CC002F08831380
:100EAE00C400C501C601C7014708CB004608CA00E9
:100EBE004508C9004408C8000A168A15E0260A1219
:100ECE008A11831203134B08C3004A08C200490853
:100EDE00C1004808C0004308CF004208CE004108B8
:100EEE00CD004008CC003B08CB003A08CA003908B8
:100EFE00C9003808C8000A168A1165220A128A111A
:100F0E00831203134B08BF004A08BE004908BD00F8
:100F1E004808BC004308CF004208CE004108CD006F
:100F2E004008CC003F08CB003E08CA003D08C9006F
:100F3E003C08C8000A168A15E0260A128A11831286
:100F4E00031348083802C4003908C5004908031CB9
:100F5E00490FC5023A08C6004A08031C4A0FC602CA
:100F6E003B08C7004B08031C4B0FC7024708B700CE
:100F7E004608B6004508B5004408B4003308CF0053
:100F8E003208CE003108CD003008CC004308CB002B
:100F9E004208CA004108C9004008C8000A168A1152
:100FAE0065220A128A118312031337084B02031D9E
:100FBE00EA2F36084A02031DEA2F35084902031D9F
:100FCE00EA2F340848020318ED2FEE2FF22FAE0150
:100FDE000314AE0DF72F0310003003180130AE00CE
:100FEE003C0883132E07FF3EAD002D08FE2F080090
:10100000A6008316031387170713181218158312E7
:101010000313AB010314AB0D2408AA002308A90095
:101020002208A8002108A700260883130A128A11A3
:1010300017270A128A158316031399000C128C12B3
:101040004528831603131813831203131813562805
:10105000831603131814181783120313181756282E
:1010600083160313181783120313181756288316B1
:101070000313181783120313181756288316031324
:101080001813831203131813562883120313250809
:101090008313013A03193028023A03193728073A13
:1010A00003192128013A031928283E2898171816F1
:1010B000831603139812981619085E28080000304A
:1010C000DB000030DC000030DD005930DF00523042
:1010D0000A168A114D210A128A1583120313D800A9
:1010E0005A30DF0055300A168A114D210A128A152E
:1010F00083120313DE005E08D806DA08031D812878
:101100008628D908031D852886288D285B08D200EB
:101110005C08D3005D08D400FE285A0883137B3E88
:10112000DE005E08D9070730DA00521C982899289B
:10113000A7285508DB07560803110318560A031D94
:10114000DC07570803110318570A031DDD07013098
:101150000310D40CD30CD20CFF3E031DA828013081
:101160000310D50DD60DD70DFF3E031DB02801305D
:10117000DA02031DBC28BD2895280930DA00521C6C
:10118000C228C328D1285508DB07560803110318C5
:10119000560A031DDC07570803110318570A031DDD
:1011A000DD0701300310D40CD30CD20CFF3E031D1D
:1011B000D22801300310DD0CDC0CDB0CFF3E031DDC
:1011C000DA280130DA02031DE628E728BF2859088B
:1011D0008313DF005B300A128A1551220A128A1526
:1011E00083120313D808031DF628F728DD175B08C0
:1011F000D2005C08D3005D08D400FE28080045300A
:10120000CA004A08CE004208CB004308CC0044087C
:10121000CD000A168A1107200A128A1583120313B9
:10122000C61F132914293B290030CE000030CF00FF
:101230000030D0004208CB004308CC004408CD0069
:101240000A168A15B6270A128A1503182829292989
:101250003229831203130030C2008030C300BF3034
:10126000C400A229831203130030C2000030C3005F
:101270000030C400A22900304602031D4129153068
:101280004502031C442945294629A2294208CB00CE
:101290004308CC004408CD000A168A113E230A12E6
:1012A0008A15831203134E08CE004D08CD004C085A
:1012B000CC004B08CB000A168A112C240A128A157E
:1012C000831203134B08C7004C08C8004D08C9001F
:1012D0004708CE004808CF004908D0004208CB009C
:1012E0004308CC004408CD000A168A15B6270A1216
:1012F0008A1503187C297D2999298312031300304C
:10130000D5008030D600BF30D7004708D20048084B
:10131000D3004908D4000A128A1530240A128A150B
:10132000831203135208C2005308C3005408C400B8
:10133000A229831203134708C2004808C3004908C2
:10134000C400A2290800A5007708FF3EA6002508D2
:101350002602A40024088313013A031DB029B129F1
:10136000C029D030A600FF30A7002508D73E840052
:1013700000082607A20027080318270AA300502AFE
:101380002408023A031DC529C629F5290A30D400CC
:101390000030D500D030A600FF30A7002508D73E8A
:1013A000840000082607D20027080318270AD30064
:1013B0000A168A15F4250A128A15831203132508C2
:1013C0008313013ED73E840000085207A800003076
:1013D000031801305307A9002808D03EA2002908AD
:1013E0000318013EFF3EA300502A2408033A031DC0
:1013F000FA29FB294B2A6430D4000030D500D030C4
:10140000A600FF30A7002508D73E84000008260765
:10141000D20027080318270AD3000A168A15F425D4
:101420000A128A158312031325088313023ED73E3E
:10143000840000085207A80053080318530AA900A3
:101440000A30D4000030D500D030AA00FF30AB0005
:101450002508013ED73E840000082A07D2002B0849
:1014600003182B0AD3000A168A15F4250A128A15C6
:101470008312031352082807AC0053080318530AB9
:101480002907AD002C08D03EA2002D080318013E0C
:10149000FF3EA300502AFF30A200FF30A300502AD5
:1014A0000800E000DF08031D562A682A600884004F
:1014B00083130008E100840A0008E200840A00089F
:1014C000E300630862046104031D672A682A742A22
:1014D00060088400003083138000840A003080009C
:1014E000840A00308000262B872A0130E100610841
:1014F000DF07600884000130E100840A840A0310D9
:10150000800C8403800C8403800CE10B7D2A003066
:10151000E1000030E200FE30E300600884000008D3
:10152000E400840A0008E500840A0008E600640874
:10153000E1056508E2056608E305630862046104E5
:10154000031DA32AA42A752AC62A0130E1006108D6
:10155000DF076008840001308007840A0030031828
:10156000013E031D8007840A00300318013E8007F6
:10157000600884000130E100840A840A0310800CB2
:101580008403800C8403800CE10BBC2A0030E10052
:101590000030E200FF30E300600884000008E4004F
:1015A000840A0008E500840A0008E6006408E105F2
:1015B0006508E2056608E305630862046104031D2B
:1015C000E22AE32AA52AF22A0130DF026008840019
:1015D0000130E1000310800D840A800D840A800D23
:1015E000E10BEA2A600884000008E100840A000890
:1015F000E200840A0008E300E21FFF2A002BE42A2D
:101600005F18032B042B0E2B60088400FF3080052D
:10161000840A7F308005840AFF3080050310DF0CC8
:101620005F08E100E201E30110300310E10DE20D7B
:10163000E30DFF3E031D152B600884006108800444
:10164000840A62088004840A630880040800031086
:10165000003003180130B60000303206031D362B6F
:1016600000303106031D362B00303006031D392BA8
:101670003A2B5E2B3308CE003408CF003508D0005B
:101680000030CB000030CC000030CD000A168A15A7
:10169000B6270A128A15031C4E2B4F2B552B2130CF
:1016A00083120313E8000030E900831203130030B3
:1016B000B0000030B1000030B2002F2C00303506F1
:1016C000031D682B00303406031D682B00303306E1
:1016D000031D6B2B6C2B732B0030B0008030B100DE
:1016E0003F30B2002F2C0030CE000030CF00003051
:1016F000D0003008CB003108CC003208CD000A16EB
:101700008A15B6270A128A150318872B882BE12B16
:10171000831203133308CB003408CC003508CD0006
:101720000A168A113E230A128A15831203134E08E1
:10173000BA004D08B9004C08B8004B08B7003A0889
:10174000BF003908BE003808BD003708BC000A16C3
:101750008A11A7200A128A158312031335083E0640
:10176000031DB82B34083D06031DB82B33083C0677
:101770000319BB2BBC2BC72B2130E8000030E9003C
:101780000030B0000030B1000030B2002F2C37081C
:101790008313B6000130BB003B08B6053008D80003
:1017A0003108D9003208DA000A168A158A240A128A
:1017B0008A15831203135808B0005908B1005A085B
:1017C000B200831203133008BC003108BD00320898
:1017D000BE000A128A1165220A128A1583120313A7
:1017E0003C08D2003D08D3003E08D4003308D500A1
:1017F0003408D6003508D7000A128A155F200A126D
:101800008A15831203135208BC005308BD00540804
:10181000BE000A128A1550250A128A158312031374
:101820003C08B0003D08B1003E08B200B608031DF8
:101830001A2C2E2C3008D8003108D9003208DA00D2
:101840000A168A158A240A128A1583120313580865
:10185000B0005908B1005A08B2002F2C2F2C0800F4
:10186000312C5C30DF0052300A168A114D210A12E9
:101870008A1583120313DA00DC08031D402C412C67
:10188000482C5508D2005608D3005708D4004F2DD5
:101890005B30DF0055300A168A114D210A128A1575
:1018A00083120313D800DB08031D572C3D2D06308F
:1018B000D9005B0883135C0203185F2C602C9F2CFB
:1018C0005B08DD005C08DD0219305D02031C692C39
:1018D0006A2C752C0030D2000030D3000030D400C8
:1018E0005B08DC005808DA009E2C01300310D50D8F
:1018F000D60DD70DFF3E031D762C0130DB025B08B1
:101900005C060319842C852C8B2C0130D902031D15
:101910008A2C8B2C752C982C01300310D40CD30CF2
:10192000D20CFF3E031D8D2C0130DD005D08DC076D
:101930005C085B06031D9D2C9E2C8C2CDF2C5C0808
:101940005B060319A42CA52CDF2C5C08DD005B08CA
:10195000DD0219305D02031CAE2CAF2CB62C00301A
:10196000D5000030D6000030D700DF2C0130031046
:10197000D20DD30DD40DFF3E031DB72C0130DC0278
:101980005B085C060319C52CC62CCC2C0130D9028F
:10199000031DCB2CCC2CB62CD92C01300310D70C2A
:1019A000D60CD50CFF3E031DCE2C0130DD005D08AA
:1019B000DB075C085B06031DDE2CDF2CCD2CDA0870
:1019C000031DE32CF72CFF30D206FF30D306FF3087
:1019D000D4060130D207003003110318013E031D65
:1019E000D307003003110318013E031DD407D808A4
:1019F000031DFB2C0F2DFF30D506FF30D606FF3020
:101A0000D7060130D507003003110318013E031D2E
:101A1000D607003003110318013E031DD70703103A
:101A2000003003180130DA005508D20756080311B8
:101A30000318560A031DD307570803110318570A42
:101A4000031DD407D41F252D262D3D2DFF30D20692
:101A5000FF30D306FF30D4060130D2070030031127
:101A60000318013E031DD307003003110318013E84
:101A7000031DD407DA010314DA0D5C088313DF00B9
:101A800052300A128A1551220A128A158312031340
:101A9000DA08031D4C2D4E2D8030D4064F2D080042
:101AA00000303E06031D5A2D00303D06031D5A2D01
:101AB00000303C06031D5D2D5E2D652D0030BC0001
:101AC0008030BD003F30BE009C2E3C08CE003D085B
:101AD000CF003E08D0007230CB003130CC00443013
:101AE000CD000A168A15B6270A128A150318792D11
:101AF0007A2D872D223083120313E8000030E9008D
:101B0000FF30BC007F30BD007F30BE009C2E8312B2
:101B100003134930CE003A30CF00C430D0003C0827
:101B2000CB003D08CC003E08CD000A168A15B6272A
:101B30000A128A1503189D2D9E2DAB2D223083127B
:101B40000313E8000030E9000030BC000030BD00A5
:101B50000030BE009C2E831203130030CE000030F4
:101B6000CF000030D0003C08CB003D08CC003E0840
:101B7000CD000A168A15B6270A128A150030031CF2
:101B8000013083120313BF00BF08031DC82DDB2DD6
:101B90003C08D8003D08D9003E08DA000A168A152C
:101BA0008A240A128A15831203135808BC005908A4
:101BB000BD005A08BE00AA30D500B830D6003F306C
:101BC000D7003C08D2003D08D3003E08D4000A12DA
:101BD0008A155F200A128A15831203135208BC006B
:101BE0005308BD005408BE003C08C2003D08C300B5
:101BF0003E08C4000A128A15FF200A128A158312B1
:101C000003134208CB004308CC004408CD000A1659
:101C10008A113E230A128A15831203134B08C0014E
:101C2000C0074C08C101C1074008C201C2074108F2
:101C3000C301C3070A168A1157200A128A15831294
:101C400003134208C5004308C6004408C7003C0807
:101C5000C2003D08C3003E08C4000A168A15482584
:101C60000A128A15831203134208BC004308BD0000
:101C70004408BE000930C7000030C8000C30C50061
:101C80000630C6003C08C2003D08C3003E08C40040
:101C90000A168A1162270A128A1583120313420850
:101CA000C2004308C3004408C4004008C501C5077A
:101CB0004108C601C6070A168A11CD260A128A15DE
:101CC000831203134208BC004308BD004408BE0051
:101CD000BF08031D6C2E9B2E7F303E06031D762E03
:101CE0007F303D06031D762EFF303C06031D792E06
:101CF0007A2E812E0030BC000030BD000030BE00C6
:101D00009C2E3C08C5003D08C6003E08C7000030B8
:101D1000C2008030C3003F30C4000A168A112D254E
:101D20000A128A15831203134208BC004308BD003F
:101D30004408BE009C2E9C2E08007C30A200063079
:101D4000A3000A168A15CF250A128A15C52FC62E9A
:101D50000A168A156B240A128A1583120313A1002E
:101D60002108F80078080A168A15F5240A128A153F
:101D7000831203137808A1007708D73E84008313E9
:101D8000210880000130A1002108F70778080D3AEA
:101D9000031DCB2ECC2EA82E0A30A4000030A500A7
:101DA000E230A2000630A30083160313D7300A16D0
:101DB0008A11F7200A128A158312031323082204BA
:101DC000031DE32EE42EF42E0A300A128A15A321F5
:101DD0000A128A15831203132208A20000300A1681
:101DE0008A15A4260A128A150A3083120313A40046
:101DF0000030A500D730A2000630A30083160313DD
:101E0000D7300A168A11F7200A128A158312031393
:101E100023082204031D0D2F0E2F1E2F0A300A1235
:101E20008A15A3210A128A15831203132208A2001D
:101E300001300A168A15A4260A128A150830831260
:101E40000313A4000030A500F630A2000630A30062
:101E500083160313D7300A168A11F7200A128A153F
:101E60008312031323082204031D372F382F622FF8
:101E7000D330A2008030A3000A168A15CF250A129B
:101E80008A15BF3083120313A2000630A3000A167E
:101E90008A15CF250A128A1500300A168A15AB2535
:101EA0000A128A150A168A1140260A128A1510305B
:101EB00083120313A2000730A3000A168A15CF2548
:101EC0000A128A15083083120313A4000030A500FB
:101ED000ED30A2000630A30083160313D7300A1694
:101EE0008A11F7200A128A15831203132308220489
:101EF000031D7B2F7C2FA62FD330A2008030A300A0
:101F00000A168A15CF250A128A15CB3083120313BD
:101F1000A2000630A3000A168A15CF250A128A15D8
:101F200001300A168A15AB250A128A150A168A117B
:101F300040260A128A15103083120313A2000730BC
:101F4000A3000A168A15CF250A128A1503108312D8
:101F50000313003003180130F7002030A1002108DE
:101F6000F800D330A2008030A3000A168A15CF25CE
:101F70000A128A157C3083120313A2000630A300D4
:101F80000A168A15CF250A128A1504308312031304
:101F9000A4000030A5000730A2000730A30083167C
:101FA0000313D7300A168A11F7200A128A158312F2
:101FB000031323082204031DDE2FDF2FA72ED330A7
:101FC000A2008030A3000A168A15CF250A128A15AE
:101FD000493083120313A2000630A3000A168A15A3
:101FE000CF250A128A15613083120313A1008316CC
:101FF000031383120313210883160313D700080069
:10200E0000304D06031D112800304C06031D11280B
:10201E0000304B06031D1428152824284E08840072
:10202E00003083138000840A003080000030CB0023
:10203E000030CC000030CD0056284D087F39CF003F
:10204E00D001013084000310CF0DD00D840B2A284F
:10205E004E0884004F0883138000840A50088000C5
:10206E004C0D4C0D0139CF00D0014E0884004F08A5
:10207E008004840A500880044E0884008230800751
:10208E00840F00080318000ACF00FF304F078000AE
:10209E0084034D0880393F38CD00CC1356280800F4
:1020AE0043084204031D5C285D2864280030C200EA
:1020BE000030C3000030C400A6284208C800430800
:1020CE00C9000030C91BFF30CA004808C5004908C6
:1020DE00C6004A08C700C31F752876287E28C50982
:1020EE00C609C709C50A0319C60A0319C70A8E30DD
:1020FE00DF0045300A128A1551220A168A11831200
:10210E000313C31F8B288C289F284508D800460828
:10211E00D9004708DA000A168A158A240A168A1187
:10212E00831203135808C5005908C6005A08C70081
:10213E004508C2004608C3004708C400A628080088
:10214E003F083E043D043C04031DAE28AF28B628CC
:10215E000030BC000030BD000030BE00F6288E30CE
:10216E00C000C62801300310BF0CBE0CBD0CBC0C49
:10217E00FF3E031DBA280130C4004408C0070030DA
:10218E00C4000030C5000030C600FF30C7003C0858
:10219E00C4053D08C5053E08C6053F08C7054708E6
:1021AE00460445044404031DDD28DE28B9283C08F6
:1021BE00C1003D08C2003E08C30040088313DF0083
:1021CE0041300A128A1551220A168A1183120313FC
:1021DE004108BC004208BD004308BE00F6280800B6
:1021EE0083120313A60036292608840083130008E1
:1021FE00003A03190329042916292208840023080A
:10220E000A128A1100260A168A11A70026088400CF
:10221E008313000827060319152916292B292208CE
:10222E00840023080A128A1100260A168A11A700B2
:10223E002608840083130008A80027082802A2009D
:10224E00A301031CA3034C290130A7002708A607EE
:10225E000130A2070318A30AA700A71BA30383122A
:10226E000130A4020030031CA503A502FF30250691
:10227E00031D4329FF302406031D46294729FB2849
:10228E000030A2000030A3004C290800E0006008D6
:10229E00840083130008E200840A0008E300840A25
:1022AE000008E4000F300310E40CE30CE20CFF3ED8
:1022BE00031D5A296208E100E5005F0884006508E5
:1022CE008000E108031D6C296D29792960088400BE
:1022DE0000308000840A00308000840A00308000C4
:1022EE000030A6290310003003180130E100600809
:1022FE00840000308004840A80308004840A003018
:10230E008004600884000008E200840A0008E300EC
:10231E00840A0008E400E41F952996299A290130C1
:10232E00E2006208E10760088400FF308005840A3D
:10233E00FF308005840A003080056108A629080058
:10234E000310003003180130AC00A91FAF29B029CB
:10235E00B829A809A909A80A0319A90AAC010314E6
:10236E00AC0DAB1FBB29BC29C129AA09AB09AA0A0E
:10237E000319AB0A2B082A040319C629C729F72902
:10238E00AD010314AD0DD62901300310AA0DAB0D0E
:10239E00FF3E031DCC290130AE002E08AD07AB1F4A
:1023AE00D929DA29CB292B082902031DE0292A086D
:1023BE002802031CE329E429EA292A08A8022B088B
:1023CE00031CA903A90201300310AB0CAA0CFF3E9B
:1023DE00031DEB290130AD02031DF629F729DA2979
:1023EE00AC08031DFB29002AA809A909A80A03198C
:1023FE00A90A012A08008312031386120F300A1647
:10240E008A152C250A168A118312031386150615B2
:10241E00861006100A168A157A240A168A110530B5
:10242E000A168A152C250A168A110A168A157A2476
:10243E000A168A11213083120313A100272A272A94
:10244E000130A102031D2C2A2D2A262A0A168A15CE
:10245E007A240A168A1105300A168A152C250A16B0
:10246E008A118312031386110A168A157A240A1604
:10247E008A110D3083120313A200462A462A013018
:10248E00A202031D4B2A4C2A452A28300A168A1509
:10249E0088250A168A1108300A168A1588250A1602
:1024AE008A110C300A168A1588250A168A110630EA
:1024BE000A168A1588250A168A1108000030D400DB
:1024CE000030D3000030D2000030D1004F084E044F
:1024DE004D044C040319742A752AC32AD00103141F
:1024EE00D00D862A0130D5000310CC0DCD0DCE0DAA
:1024FE00CF0DD50B7B2A0130D5005508D007CF1F45
:10250E00892A8A2A792A0130D5000310D10DD20DDD
:10251E00D30DD40DD50B8C2A4F084B02031DA12AC7
:10252E004E084A02031DA12A4D084902031DA12A85
:10253E004C084802031CA42AA52AB42A4C08C80237
:10254E004D08031C4D0FC9024E08031C4E0FCA0244
:10255E004F08031C4F0FCB02511401300310CF0C48
:10256E00CE0CCD0CCC0CFF3E031DB52A0130D00293
:10257E00031DC22AC32A8A2A5408CB005308CA0054
:10258E005208C9005108C800CC2A080003100030B8
:10259E0003180130AC00AB1FD52AD62ADE2AAA09B1
:1025AE00AB09AA0A0319AB0AAC010314AC0DA91F9F
:1025BE00E12AE22AEB2AA809A909A80A0319A90AFD
:1025CE000130B0003008AC060030AE000030AF0075
:1025DE002B082A040319F42AF52A2D2BAD01031416
:1025EE00AD0D042B01300310AA0DAB0DFF3E031DE4
:1025FE00FA2A0130B0003008AD07AB1F072B082BAD
:10260E00F92A01300310AE0DAF0DFF3E031D092B4D
:10261E002B082902031D152B2A082802031C182B30
:10262E00192B202B2A08A8022B08031CA903A90288
:10263E002E1401300310AB0CAA0CFF3E031D212BF0
:10264E000130AD02031D2C2B2D2B082BAC08031DC6
:10265E00312B362BAE09AF09AE0A0319AF0A2E087D
:10266E00A801A8072F08A901A9073D2B0800503083
:10267E00DF004B300A168A114D210A168A11831279
:10268E000313CF004B08D1004C08D2004D08D300E5
:10269E00D4018E30D002D01F552B562B792B5008DB
:1026AE008313803A8F3E03185D2B5E2B672B003011
:1026BE00CE000030CD000030CC000030CB00B12B6E
:1026CE0001300310D40CD30CD20CD10CFF3E031DE1
:1026DE00682B0130D5005508D007031D772B782BBA
:1026EE00672B992B20305002031C7E2B7F2B882BBF
:1026FE000030CE000030CD000030CC000030CB00DA
:10270E00B12B942B0130D5000310D10DD20DD30D6A
:10271E00D40DD50B8B2B0130D002D008031D982B76
:10272E00992B892BCF08031D9D2BA82BD109D209DC
:10273E00D309D409D10A0319D20A0319D30A0319EA
:10274E00D40A5408CE005308CD005208CC005108CC
:10275E00CB00B12B08006A08C201C2076B08C30187
:10276E00C3070A168A1157200A168A1183120313F9
:10277E004208A1004308A2004408A3002108C20099
:10278E002208C3002308C4000030C5000030C60074
:10279E004030C7000A168A112D250A168A11831297
:1027AE0003134208A4004308A5004408A600240809
:1027BE00CB002508CC002608CD000A168A113E2330
:1027CE000A168A11831203134E08AA004D08A90097
:1027DE004C08A8004B08A7000030CF000030CE00F8
:1027EE000630CD004030CC002A08CB002908CA00A4
:1027FE002808C9002708C8000A168A15E0260A16F6
:10280E008A11831203134B08F6004A08F500490893
:10281E00F4004808F3007C08AB00AC01AD01AE013A
:10282E002B08F3072C08031103182C0A031DF407B9
:10283E002D08031103182D0A031DF5072E08031189
:10284E0003182E0A031DF60708004E084D044C040B
:10285E004B04031D332C342C3B2C0030CB000030AA
:10286E00CC000030CD00A92C03100030031801302D
:10287E00CF00CE1F432C442C522CCB09CC09CD09B2
:10288E00CE09CB0A0319CC0A0319CD0A0319CE0AB5
:10289E00CF010314CF0D8E30D000622C0130031007
:1028AE00CE0CCD0CCC0CCB0CFF3E031D562C0130A8
:1028BE00D4005408D0070030D4000030D5000030CA
:1028CE00D600FF30D7004B08D4054C08D5054D086F
:1028DE00D6054E08D7055708560455045404031D53
:1028EE00792C7A2C552C4B08D1004C08D2004D086F
:1028FE00D30050088313DF0051300A128A1551227B
:10290E000A168A1183120313CF08031D8F2CA22CD3
:10291E005108D8005208D9005308DA000A168A1551
:10292E008A240A168A11831203135808D1005908F3
:10293E00D2005A08D3005108CB005208CC005308DD
:10294E00CD00A92C08000310003003180130AD0093
:10295E000430AF00B22CC72C1030B0002730B100BD
:10296E00D62CE830B0000330B100D62C6430B00065
:10297E000030B100D62C0A30B0000030B100D62C99
:10298E002F088313013A0319C22C033A0319BD2CE5
:10299E00013A0319B82C073A0319B32CD62C300878
:1029AE00B601B6073108B701B7072B08B401B40753
:1029BE002C08B501B5070A168A156C270A168A1156
:1029CE00831203133408AE00AD08031DEF2CF02C58
:1029DE00F42CAE08031DF42C012D2E088313303E6B
:1029EE000A168A1549240A168A1183120313AD0199
:1029FE000314AD0D3008D401D4073108D501D50725
:102A0E002E088313B200B3013208D2003308D3006C
:102A1E000A168A15F4250A168A1183120313520810
:102A2E00AB025308031CAC03AC020130AF02013001
:102A3E002F020318232D242DB22C2B088313303E86
:102A4E000A168A1549240A168A1108000030CC008D
:102A5E000030CD000030CE004A30DF0042300A1682
:102A6E008A114D210A168A1183120313C900CA084E
:102A7E00031D422D432D4A2D4C08C2004D08C300A4
:102A8E004E08C400B32D4830DF0045300A168A11B7
:102A9E004D210A168A1183120313CB00C808031D99
:102AAE00592D5A2D612D4C08C2004D08C3004E08F9
:102ABE00C400B32D48088313893ECF004F08CA02C5
:102ACE004B08CF004F08C9061830CB000130031059
:102ADE00CC0DCD0DCE0DFF3E031D6E2D47084402CD
:102AEE00031D7F2D46084302031D7F2D450842021C
:102AFE00031C822D832D8E2D4508C2024608031C11
:102B0E00460FC3024708031C470AC4024C14013087
:102B1E000310C20DC30DC40DFF3E031D8F2D0130DA
:102B2E00CB02031D9B2D9C2D6D2D4A088313DF00B8
:102B3E004C300A128A1551220A168A118312031377
:102B4E00C908031DAB2DAC2DCE174C08C2004D0885
:102B5E00C3004E08C400B32D08000030CF00003073
:102B6E00CE000030CD006430CC007608CB00750866
:102B7E00CA007408C9007308C8000A168A116522B3
:102B8E000A168A11831203134B08CB004A08CA0097
:102B9E004908C9004808C8002208CC002308CD0007
:102BAE000030CD1BFF30CE00CF000A168A15E0266E
:102BBE000A168A11831203134B08EF004A08EE001F
:102BCE004908ED004808EC00603083160313D50069
:102BDE00EA30D600352E04308706831603135508C7
:102BEE00B03E83120313A400831603135608031872
:102BFE00013E043E83120313A500F6302502031D89
:102C0E000A2E1830240203180D2E0E2E2C2E83168B
:102C1E000313B030D5070318D60A0430D607831233
:102C2E00031383160313550883120313A601A60775
:102C3E0083160313560883120313A701A7070A1658
:102C4E008A1548260A168A11352EFF30A600FF3047
:102C5E00A7000A168A1548260A168A11831203132C
:102C6E006F086E046D046C04031D3E2E3F2EF22D74
:102C7E00080083120313A4006430AA000030AB00D6
:102C8E0024088313A600A7012608A8002708A90078
:102C9E000A168A11CD220A168A11831203132808E6
:102CAE00A801A8072908A901A9070A30AA0000301F
:102CBE00AB000A168A11A7210A168A118312031372
:102CCE002808A5000A30AA000030AB0024088313A0
:102CDE00A600A7012608A8002708A9000A168A112F
:102CEE00CD220A168A11831203132808A801A807F9
:102CFE002908A901A9070A30AA000030AB000A165C
:102D0E008A11A7210A168A11831203132808A2001A
:102D1E000A30AA000030AB0024088313A600A701D6
:102D2E002608A8002708A9000A168A11A7210A1644
:102D3E008A11831203132808A300A508031DA82EC9
:102D4E00A92EB02E20300A168A15F5240A168A11DD
:102D5E00B82E25088313303E0A168A15F5240A1656
:102D6E008A118312031322088313303E0A168A1522
:102D7E00F5240A168A118312031323088313303E97
:102D8E000A168A15F5240A168A1108000030440620
:102D9E00031DD72E00304306031DD72E00304206EA
:102DAE00031DDA2EDB2EE22E0030C2000030C300EF
:102DBE000030C400612F44087F39C700C8010130BC
:102DCE0084000310C70DC80D840BE82E4708C507F5
:102DDE000318C60A4808C607430D430D0139C7003C
:102DEE00C8014708C5070318C60A4808C607C61F04
:102DFE00012F022F0D2F2230E8000030E9000030A5
:102E0E00C2000030C3000030C400612F4608803A73
:102E1E00C70081304702031D162F00304502031CE8
:102E2E00192F1A2F452F2230E8000030E90000300C
:102E3E00CE000030CF000030D0004208CB00430857
:102E4E00CC004408CD000A168A15B6270A168A1138
:102E5E000318322F332F3C2F83120313FF30C2007F
:102E6E007F30C300FF30C400612F83120313FF3085
:102E7E00C2007F30C3007F30C400612F4608C800F7
:102E8E004508C7000130C900480DC80CC70CC90B56
:102E9E004B2F4408470680394706C4004508831364
:102EAE000139C700C70CC70C430847067F394706D0
:102EBE00C300612F08004608D0004508CF0003303C
:102ECE00D200470883130A168A1510250A168A118E
:102EDE00831203134F07840050080318500AD100C1
:102EEE000A128A1100260A168A11CC00840A0319C6
:102EFE00D10A51080A128A1100260A168A11CD002B
:102F0E00840A0319D10A51080A128A1100260A16D8
:102F1E008A11CE00F22F4C08D5004D08D6004E086F
:102F2E00D7004208D2004308D3004408D4000A1246
:102F3E008A155F200A168A11831203135208C900DC
:102F4E005308CA005408CB004608D0004508CF00ED
:102F5E000330D200FF30C7070318C80AFF30C80776
:102F6E0047080A168A1510250A168A1183120313AA
:102F7E004F07840050080318500AD1000A128A1114
:102F8E0000260A168A11D500840A0319D10A51089F
:102F9E000A128A1100260A168A11D600840A03190B
:102FAE00D10A51080A128A1100260A168A11D70070
:102FBE004908D2004A08D3004B08D4000A128A15D9
:102FCE0030240A168A11831203135208CC005308B8
:102FDE00CD005408CE0048084704031DF72FF82FE4
:102FEE00922F4C08C2004D08C3004E08C400FF2F9C
:022FFE000800C9
:10389200B400861634080A168A1588250A168A156F
:1038A200080083120313AD0086122D0883130A1633
:1038B2008A1588250A168A15080001300A168A1503
:1038C20052240A168A1503300A168A152C250A165E
:1038D2008A150800712C0A168A15C5240A168A153B
:1038E200831203138C1E762C772C6C2C1A08792CDD
:1038F2000800831203130616B8010314B80D822CB4
:10390200822C0130B802031D872C882C812C0612D0
:10391200080000305A06031D942C00305906031D7E
:10392200942C003058060319972C982C9A2C80302E
:10393200DA069B2C0800163083120313A90000300C
:10394200AA00051EA52CA62CAE2C05080F39AB002B
:10395200AC012B08A9002C08AA00AF2C0800A1007A
:103962002118B42CB82C831203138714BB2C831296
:10397200031387106430A2000030A3000A168A11D4
:10398200B4250A168A150800981CC82CC92CD12CFB
:10399200831603139812981683120313181218161B
:1039A200181DD42CD52CDB2C1A08AA00831603135D
:1039B2009812981608002118DF2CE32C83120313A7
:1039C2008714E62C83120313871004308706FF3016
:1039D2008F007D088E001014EE2C0C1CF12CF22CA2
:1039E200EE2C0C1010100800A800FC2C0A168A15E8
:1039F200C5240A168A15831203130C1E012D022DEB
:103A0200F72C2808831399001530A900092D092DD8
:103A12000130A902031D0E2D0F2D082D0800D30021
:103A22000310003003180130D400531C192D1A2D35
:103A32001F2D52088313D5005508D4070310D20D49
:103A42000310D30CD308031D272D282D162D54083F
:103A520083132B2D080083120313AB000430AC0038
:103A62005330AD00352D352D0130AD02031D3A2DF9
:103A72003B2D342D0130AC02031D402D412D312D43
:103A82000130AB02031D462D472D2F2D080080303B
:103A9200C7064508D5004608D6004708D7004208A1
:103AA200D2004308D3004408D4000A128A153024F5
:103AB2000A168A15831203135208C2005308C30060
:103AC2005408C400642D0800B700B71F692D6A2D81
:103AD2006C2D06146D2D0610371F702D712D732D50
:103AE2008614742D8610B71E772D782D7A2D061523
:103AF2007B2D0611371E7E2D7F2D812D8615822D61
:103B020086110A168A157A240A168A150800831263
:103B12000313B500350883130A168A1565250A169C
:103B22008A1583120313B50EF030B50535088313D9
:103B32000A168A1565250A168A151130831203138F
:103B4200B600A42DA42D0130B602031DA92DAA2D65
:103B5200A32D080083120313A200B02DB02D8316EB
:103B620003178C18B52DB62DAF2D8312031322081F
:103B72008313831203178D007F3083120313A30074
:103B820083160317831203132308831603178C0566
:103B92000C14831203170C08CE2D0800E62D220800
:103BA200840023080A128A1100260A168A150A16A8
:103BB2008A15F5240A168A15013083120313A20707
:103BC2000318A30AA400A41BA30322088400230849
:103BD2000A128A1100260A168A150038031DF22DD0
:103BE200F32DD02D08000030D6000030D700521C33
:103BF200FB2DFC2D022E5408D6070318D70A5508B0
:103C0200D70701300310D40DD50DFF3E031D032E3F
:103C120001300310D30CD20CFF3E031D0A2E5308B1
:103C22005204031D152E162EF82D5608D201D20766
:103C32005708D301D3071D2E08000830AB0001300E
:103C42000A168A1572260A168A1583120313290880
:103C5200AB01AB072A08AC01AC070A168A11AA24E9
:103C62000A168A150C3083120313AB000730AC001E
:103C72000A128A113F220A168A1583120313871128
:103C820014300A168A152C250A168A1508000130E6
:103C9200A8000030A9000030AA000030AB002808BC
:103CA200EC022908031C290F572E582EED022A0870
:103CB200031C2A0F5D2E5E2EEE022B08031C2B0F17
:103CC200632E642EEF0227088F00260883138E00CE
:103CD20010146B2E0C1C6E2E6F2E6B2E0C101010EF
:103CE2000800AC00942E2B087F3E0A168A15522437
:103CF2000A168A15A32E2B08BF3E0A168A155224CD
:103D02000A168A15A32E2B08933E0A168A155224E8
:103D12000A168A15A32E2B08D33E0A168A15522498
:103D22000A168A15A32E2C088313013A0319742E3E
:103D3200033A03197C2E013A0319842E073A031918
:103D42008C2EA32E0800A300A72EA72E83160317DE
:103D52008C18AC2EAD2EA62E8312031323088313C8
:103D6200831203178D008312031322088312031791
:103D72008C007F3083120313A4008316031783126F
:103D820003132408831603178C05831203130310ED
:103D92008B1FCC2ECD2ECE2E03148B13831603171E
:103DA2000C1555308D00AA308D008C140C11831225
:103DB2000313031CDD2EDE2EDF2E8B1708000030CE
:103DC200D3000030D2000030D1000030D000481CB7
:103DD200EB2EEC2E002F4C08D0074D0803110318D0
:103DE2004D0A031DD1074E08031103184E0A031D85
:103DF200D2074F08031103184F0A031DD3070130DE
:103E0200D4000310CC0DCD0DCE0DCF0DD40B022F4F
:103E120001300310CB0CCA0CC90CC80CFF3E031DA9
:103E22000A2F4B084A0449044804031D192F1A2F6C
:103E3200E82E5308CB005208CA005108C9005008A6
:103E4200C800232F08002908C201C2072A08C3019B
:103E5200C3070A168A1157200A168A1583120313FA
:103E62004208AD004308AE004408AF002B08C2016F
:103E7200C2072C08C301C3070A168A1157200A1663
:103E82008A15831203134208B3004308B40044089E
:103E9200B5002D08B0002E08B1002F08B2000A129A
:103EA2008A1527230A168A15831203133008CB00BA
:103EB2003108CC003208CD000A168A113E230A16B8
:103EC2008A15831203134B08A901A9074C08AA01FA
:103ED200AA076B2F08000030B9000030BA0037087B
:103EE20036040319752F762FAE2FB8010314B80DBF
:103EF200852F01300310B60DB70DFF3E031D7B2F3A
:103F02000130BB003B08B807B71F882F892F7A2FD3
:103F120001300310B90DBA0DFF3E031D8A2F370879
:103F22003502031D962F36083402031C992F9A2F4F
:103F3200A12F3608B4023708031CB503B5023914A1
:103F420001300310B70CB60CFF3E031DA22F013047
:103F5200B802031DAD2FAE2F892F3908B401B40763
:103F62003A08B501B507B52F0800CD1FB92FBA2FF2
:103F7200D02F0030D1000030D2008030D3004B0867
:103F8200D1024C080318D203D2024D080318D303FE
:103F9200D3025108CB005208CC005308CD00D01FE9
:103FA200D32FD42FEA2F0030D1000030D20080303E
:103FB200D3004E08D1024F080318D203D202500890
:103FC2000318D303D3025108CE005208CF0053087E
:103FD200D0008030CD068030D00650084D02031D3F
:103FE200F82F4F084C02031DF82F4E084B020318FE
:0E3FF200FB2FFD2F0314FE2F0310FF2F0800DE
:00000001FF
